:1000000010C01FC01EC01DC01CC01BC01AC019C01C
:1000100018C050C05EC06CC014C013C012C011C064
:1000200010C011241FBECFE5D1E0DEBFCDBF10E070
:10003000A0E6B0E001C01D92A236B107E1F755D1AC
:10004000A6C1DECF91B1976091B9877087B983EC73
:1000500086B93699FECF24B135B116B8C9010895D5
:10006000813099F4623019F4D89AD99804C061307B
:1000700029F4D99AD8986093610008958BB38C7F46
:100080008BBB8FEF809361000895823091F46230D2
:1000900019F4DA9ADB9804C0613029F4DB9ADA9813
:1000A0006093600008958BB3837F8BBB8FEF809349
:1000B000600008951F920F920FB60F9211248F9334
:1000C0008BB38C7F8BBB8F910F900FBE0F901F90C7
:1000D00018951F920F920FB60F9211248F938BB326
:1000E000837F8BBB8F910F900FBE0F901F90189541
:1000F0001F920F920FB60F9211242F933F934F939D
:100100005F936F937F938F939F93AF93BF93EF937F
:10011000FF936091610081E0A3DF6091600082E065
:100120009FDFFF91EF91BF91AF919F918F917F9151
:100130006F915F914F913F912F910F900FBE0F9054
:100140001F90189582E083BF83E080BF87E089BF5E
:100150008FE786BF86B78CBF12BE08958BB38C7FA6
:100160008BBB8AB383608ABB8BB3837F8BBB8AB321
:100170008C608ABB08951F93982F162F8091610081
:10018000891719F081E0692F6BDF8091600081177A
:1001900019F082E0612F64DF1F910895813011F41E
:1001A00086B708958CB70895982F86B7891396BFA0
:1001B0008CB786136CBF08952AEF30E004C0F901B4
:1001C0003197F1F701970097D1F708954AEF50E082
:1001D0001AC0FA013197F1F7215030409FEF2F3FBD
:1001E0003907B9F7DC9AD49A22E330E003C0FA0168
:1001F0003197F1F7215030409FEF2F3F3907B9F782
:10020000DC98D49A8150882319F026EB33E0E4CFB0
:100210000895BA9AC29A8AEF90E00197F1F781B1F6
:10022000876081B987E087B983EC86B93699FECFBC
:1002300044B155B116B8C2988AEF90E00197F1F732
:1002400081B1876081B987E087B983EC86B9369937
:10025000FECF24B135B116B8241B350BC901089562
:1002600086B78E3211F08EE286BF8CB78E3211F0D7
:100270008EE28CBF81E061E07EDF2CE231E04AEF6C
:1002800050E003C0CA010197F1F7215030408FEFD1
:100290002F3F3807B9F786B78E3211F08EE286BF4E
:1002A0008CB78E3211F08EE28CBF81E062E063DFAA
:1002B0002CE231E04AEF50E003C0CA010197F1F7A8
:1002C000215030408FEF2F3F3807B9F7089586B798
:1002D000863211F086E286BF8CB7863211F086E254
:1002E0008CBF82E062E047DF0895F89429E288E15C
:1002F00090E00FB6F894A89581BD0FBE21BD8BB3D9
:100300008C7F8BBB8AB383608ABB8BB3837F8BBBB1
:100310008AB38C608ABB8FEF6FEF2DDF82E083BFE3
:1003200083E080BF87E089BF8FE786BF86B78CBF39
:1003300012BEDC9AD49A28EE33E04AEF50E003C0B4
:10034000CA010197F1F7215030408FEF2F3F380756
:10035000B9F7DC98D49A28EE33E04AEF50E003C0B6
:10036000CA010197F1F7215030408FEF2F3F380736
:10037000B9F778944EDFC39720F0DC98D49AA7DFC2
:1003800004C0DC9AD49A80E06BDFA895F3CFF89490
:02039000FFCF9D
:00000001FF
